 bytecodes001

 Timestamp is 4b0eb771 (reproducible build file hash)

 Preferred load address is 0000000180000000

 Start         Length     Name                   Class
 0001:00000000 00002bb0H .text$mn                CODE
 0001:00002bb0 00000036H .text$mn$00             CODE
 0001:00002be6 00000092H .text$x                 CODE
 0002:00000000 00000198H .idata$5                DATA
 0002:00000198 00000038H .00cfg                  DATA
 0002:000001d0 00000008H .CRT$XCA                DATA
 0002:000001d8 00000008H .CRT$XCZ                DATA
 0002:000001e0 00000008H .CRT$XIA                DATA
 0002:000001e8 00000008H .CRT$XIC                DATA
 0002:000001f0 00000008H .CRT$XIZ                DATA
 0002:000001f8 00000008H .CRT$XLA                DATA
 0002:00000200 00000008H .CRT$XLZ                DATA
 0002:00000208 00000008H .CRT$XPA                DATA
 0002:00000210 00000008H .CRT$XPZ                DATA
 0002:00000218 00000008H .CRT$XTA                DATA
 0002:00000220 00000010H .CRT$XTZ                DATA
 0002:00000228 00000000H .gehcont$y              DATA
 0002:00000228 00000000H .gfids$y                DATA
 0002:00000230 00001b50H .rdata                  DATA
 0002:00001d80 00000000H .rdata$CastGuardVftablesA DATA
 0002:00001d80 00000000H .rdata$CastGuardVftablesC DATA
 0002:00001d80 00000028H .rdata$T                DATA
 0002:00001da8 000000b0H .rdata$voltmd           DATA
 0002:00001e58 00000320H .rdata$zzzdbg           DATA
 0002:00002178 00000008H .rtc$IAA                DATA
 0002:00002180 00000008H .rtc$IZZ                DATA
 0002:00002188 00000008H .rtc$TAA                DATA
 0002:00002190 00000008H .rtc$TZZ                DATA
 0002:00002198 00000004H .tls                    DATA
 0002:0000219c 00000004H .tls$                   DATA
 0002:000021a0 00000008H .tls$ZZZ                DATA
 0002:000021a8 000002e8H .xdata                  DATA
 0002:00002490 000003a0H .edata                  DATA
 0002:00002830 00000064H .idata$2                DATA
 0002:00002894 00000014H .idata$3                DATA
 0002:000028a8 00000198H .idata$4                DATA
 0002:00002a40 0000041eH .idata$6                DATA
 0003:00000000 000000f0H .data                   DATA
 0003:000000f0 0001b248H .bss                    DATA
 0004:00000000 00000378H .pdata                  DATA

  Address         Publics by Value              Rva+Base               Lib:Object

 0000:00000000       __AbsoluteZero             0000000000000000     <absolute>
 0000:00000000       ___safe_se_handler_count   0000000000000000     <absolute>
 0000:00000000       ___safe_se_handler_table   0000000000000000     <absolute>
 0000:00000000       __arm64x_extra_rfe_table   0000000000000000     <absolute>
 0000:00000000       __arm64x_extra_rfe_table_size 0000000000000000     <absolute>
 0000:00000000       __arm64x_native_entrypoint 0000000000000000     <absolute>
 0000:00000000       __arm64x_redirection_metadata 0000000000000000     <absolute>
 0000:00000000       __arm64x_redirection_metadata_count 0000000000000000     <absolute>
 0000:00000000       __dynamic_value_reloc_table 0000000000000000     <absolute>
 0000:00000000       __enclave_config           0000000000000000     <absolute>
 0000:00000000       __guard_check_icall_a64n_fptr 0000000000000000     <absolute>
 0000:00000000       __guard_eh_cont_count      0000000000000000     <absolute>
 0000:00000000       __guard_eh_cont_table      0000000000000000     <absolute>
 0000:00000000       __guard_fids_count         0000000000000000     <absolute>
 0000:00000000       __guard_fids_table         0000000000000000     <absolute>
 0000:00000000       __guard_iat_count          0000000000000000     <absolute>
 0000:00000000       __guard_iat_table          0000000000000000     <absolute>
 0000:00000000       __guard_longjmp_count      0000000000000000     <absolute>
 0000:00000000       __guard_longjmp_table      0000000000000000     <absolute>
 0000:00000000       __hybrid_auxiliary_iat     0000000000000000     <absolute>
 0000:00000000       __hybrid_auxiliary_iat_copy 0000000000000000     <absolute>
 0000:00000000       __hybrid_code_map          0000000000000000     <absolute>
 0000:00000000       __hybrid_code_map_count    0000000000000000     <absolute>
 0000:00000000       __x64_code_ranges_to_entry_points 0000000000000000     <absolute>
 0000:00000000       __x64_code_ranges_to_entry_points_count 0000000000000000     <absolute>
 0000:00000100       __guard_flags              0000000000000100     <absolute>
 0000:00000000       __ImageBase                0000000180000000     <linker-defined>
 0001:00000000       ?NewObject@JNIEnv_@@QEAAPEAV_jobject@@PEAV_jclass@@PEAU_jmethodID@@ZZ 0000000180001000 f i libbytecodes001.obj
 0001:00000024       ?TranslateError@@YAPEBDW4jvmtiError@@@Z 0000000180001024 f   libbytecodes001.obj
 0001:000002dc       ?nsk_jni_check_exception@@YAHPEAUJNIEnv_@@QEBDH@Z 00000001800012dc f   libbytecodes001.obj
 0001:00000420       ?nsk_jni_lverify@@YAHHPEAUJNIEnv_@@HQEBDH1ZZ 0000000180001420 f   libbytecodes001.obj
 0001:000004c0       Agent_Initialize           00000001800014c0 f   libbytecodes001.obj
 0001:00000604       Agent_OnAttach             0000000180001604 f   libbytecodes001.obj
 0001:00000604       Agent_OnLoad               0000000180001604 f   libbytecodes001.obj
 0001:0000060c       Java_nsk_jvmti_GetBytecodes_bytecodes001_check 000000018000160c f   libbytecodes001.obj
 0001:00000658       Java_nsk_jvmti_unit_FollowReferences_FollowRefObjects_addRefToVerify 0000000180001658 f   libbytecodes001.obj
 0001:00000814       Java_nsk_jvmti_unit_FollowReferences_FollowRefObjects_getTag 0000000180001814 f   libbytecodes001.obj
 0001:000008d0       Java_nsk_jvmti_unit_FollowReferences_FollowRefObjects_resetRefsToVerify 00000001800018d0 f   libbytecodes001.obj
 0001:000008d8       Java_nsk_jvmti_unit_FollowReferences_FollowRefObjects_resetTags 00000001800018d8 f   libbytecodes001.obj
 0001:0000091c       Java_nsk_jvmti_unit_FollowReferences_FollowRefObjects_setTag 000000018000191c f   libbytecodes001.obj
 0001:00000b68       Java_nsk_share_jvmti_ArgumentHandler_getAgentOptionsString 0000000180001b68 f   libbytecodes001.obj
 0001:00000c14       Java_nsk_share_jvmti_DebugeeClass_checkStatus 0000000180001c14 f   libbytecodes001.obj
 0001:00000c9c       Java_nsk_share_jvmti_DebugeeClass_resetAgentData 0000000180001c9c f   libbytecodes001.obj
 0001:00000cfc       Java_nsk_share_jvmti_RedefineAgent_agentStatus 0000000180001cfc f   libbytecodes001.obj
 0001:00000d08       Java_nsk_share_jvmti_RedefineAgent_isRedefined 0000000180001d08 f   libbytecodes001.obj
 0001:00000d14       Java_nsk_share_jvmti_RedefineAgent_redefineAttempted 0000000180001d14 f   libbytecodes001.obj
 0001:00000d20       MA_checkStatus             0000000180001d20 f   libbytecodes001.obj
 0001:00000dc4       __local_stdio_printf_options 0000000180001dc4 f i libbytecodes001.obj
 0001:00000f94       checkMeth                  0000000180001f94 f   libbytecodes001.obj
 0001:00001138       exitOnError                0000000180002138 f   libbytecodes001.obj
 0001:000011ec       fprintf                    00000001800021ec f i libbytecodes001.obj
 0001:00001230       nsk_jvmti_lverify          0000000180002230 f   libbytecodes001.obj
 0001:00001320       nsk_jvmti_resetAgentData   0000000180002320 f   libbytecodes001.obj
 0001:00001394       nsk_lcomplain              0000000180002394 f   libbytecodes001.obj
 0001:000013b4       nsk_ldisplay               00000001800023b4 f   libbytecodes001.obj
 0001:000013d4       nsk_ltrace                 00000001800023d4 f   libbytecodes001.obj
 0001:000013f4       nsk_lvcomplain             00000001800023f4 f   libbytecodes001.obj
 0001:000015ac       nsk_lvdisplay              00000001800025ac f   libbytecodes001.obj
 0001:000015f8       nsk_lverify                00000001800025f8 f   libbytecodes001.obj
 0001:00001654       nsk_lvtrace                0000000180002654 f   libbytecodes001.obj
 0001:000016b4       nsk_printf                 00000001800026b4 f   libbytecodes001.obj
 0001:000016dc       nsk_vprintf                00000001800026dc f   libbytecodes001.obj
 0001:00001790       printf                     0000000180002790 f i libbytecodes001.obj
 0001:00001c90       __raise_securityfailure    0000000180002c90 f   MSVCRT:gs_report.obj
 0001:00001cc4       __report_gsfailure         0000000180002cc4 f   MSVCRT:gs_report.obj
 0001:00001f04       __GSHandlerCheck           0000000180002f04 f   MSVCRT:gshandler.obj
 0001:00001f24       __GSHandlerCheckCommon     0000000180002f24 f   MSVCRT:gshandler.obj
 0001:00001f90       __security_check_cookie    0000000180002f90 f   MSVCRT:amdsecgs.obj
 0001:000022d0       _DllMainCRTStartup         00000001800032d0 f   MSVCRT:dll_dllmain.obj
 0001:00002310       __scrt_acquire_startup_lock 0000000180003310 f   MSVCRT:utility.obj
 0001:0000234c       __scrt_dllmain_after_initialize_c 000000018000334c f   MSVCRT:utility.obj
 0001:00002380       __scrt_dllmain_before_initialize_c 0000000180003380 f   MSVCRT:utility.obj
 0001:00002398       __scrt_dllmain_crt_thread_attach 0000000180003398 f   MSVCRT:utility.obj
 0001:000023c0       __scrt_dllmain_crt_thread_detach 00000001800033c0 f   MSVCRT:utility.obj
 0001:000023d8       __scrt_dllmain_exception_filter 00000001800033d8 f   MSVCRT:utility.obj
 0001:00002438       __scrt_dllmain_uninitialize_c 0000000180003438 f   MSVCRT:utility.obj
 0001:00002468       __scrt_dllmain_uninitialize_critical 0000000180003468 f   MSVCRT:utility.obj
 0001:0000247c       __scrt_initialize_crt      000000018000347c f   MSVCRT:utility.obj
 0001:000024c8       __scrt_initialize_onexit_tables 00000001800034c8 f   MSVCRT:utility.obj
 0001:00002554       __scrt_is_nonwritable_in_current_image 0000000180003554 f   MSVCRT:utility.obj
 0001:000025ec       __scrt_release_startup_lock 00000001800035ec f   MSVCRT:utility.obj
 0001:00002610       __scrt_uninitialize_crt    0000000180003610 f   MSVCRT:utility.obj
 0001:0000263c       _onexit                    000000018000363c f   MSVCRT:utility.obj
 0001:00002678       atexit                     0000000180003678 f   MSVCRT:utility.obj
 0001:00002690       __crt_debugger_hook        0000000180003690 f   MSVCRT:utility_desktop.obj
 0001:00002698       __scrt_fastfail            0000000180003698 f   MSVCRT:utility_desktop.obj
 0001:000027e4       _guard_check_icall_nop     00000001800037e4 f i MSVCRT:guard_support.obj
 0001:000027e8       __security_init_cookie     00000001800037e8 f   MSVCRT:gs_support.obj
 0001:00002894       DllMain                    0000000180003894 f   MSVCRT:dll_dllmain_stub.obj
 0001:000028b8       ?__scrt_initialize_type_info@@YAXXZ 00000001800038b8 f   MSVCRT:tncleanup.obj
 0001:000028c8       ?__scrt_uninitialize_type_info@@YAXXZ 00000001800038c8 f   MSVCRT:tncleanup.obj
 0001:000028d4       __local_stdio_scanf_options 00000001800038d4 f i MSVCRT:default_local_stdio_options.obj
 0001:000028dc       __scrt_initialize_default_local_stdio_options 00000001800038dc f   MSVCRT:default_local_stdio_options.obj
 0001:000028f8       __scrt_get_dyn_tls_init_callback 00000001800038f8 f   MSVCRT:dyn_tls_init.obj
 0001:00002900       _RTC_Initialize            0000000180003900 f   MSVCRT:initsect.obj
 0001:0000293c       _RTC_Terminate             000000018000393c f   MSVCRT:initsect.obj
 0001:00002978       __isa_available_init       0000000180003978 f   MSVCRT:cpu_disp.obj
 0001:00002b24       _get_startup_argv_mode     0000000180003b24 f   MSVCRT:argv_mode.obj
 0001:00002b2c       __scrt_is_ucrt_dll_in_use  0000000180003b2c f   MSVCRT:ucrt_detection.obj
 0001:00002b40       memcpy                     0000000180003b40 f   vcruntime:VCRUNTIME140.dll
 0001:00002b46       memset                     0000000180003b46 f   vcruntime:VCRUNTIME140.dll
 0001:00002b4c       strchr                     0000000180003b4c f   vcruntime:VCRUNTIME140.dll
 0001:00002b52       __C_specific_handler       0000000180003b52 f   vcruntime:VCRUNTIME140.dll
 0001:00002b58       __std_type_info_destroy_list 0000000180003b58 f   vcruntime:VCRUNTIME140.dll
 0001:00002b5e       strcmp                     0000000180003b5e f   ucrt:api-ms-win-crt-string-l1-1-0.dll
 0001:00002b64       strlen                     0000000180003b64 f   ucrt:api-ms-win-crt-string-l1-1-0.dll
 0001:00002b6a       _initterm                  0000000180003b6a f   ucrt:api-ms-win-crt-runtime-l1-1-0.dll
 0001:00002b70       _initterm_e                0000000180003b70 f   ucrt:api-ms-win-crt-runtime-l1-1-0.dll
 0001:00002b76       _seh_filter_dll            0000000180003b76 f   ucrt:api-ms-win-crt-runtime-l1-1-0.dll
 0001:00002b7c       _configure_narrow_argv     0000000180003b7c f   ucrt:api-ms-win-crt-runtime-l1-1-0.dll
 0001:00002b82       _initialize_narrow_environment 0000000180003b82 f   ucrt:api-ms-win-crt-runtime-l1-1-0.dll
 0001:00002b88       _initialize_onexit_table   0000000180003b88 f   ucrt:api-ms-win-crt-runtime-l1-1-0.dll
 0001:00002b8e       _register_onexit_function  0000000180003b8e f   ucrt:api-ms-win-crt-runtime-l1-1-0.dll
 0001:00002b94       _execute_onexit_table      0000000180003b94 f   ucrt:api-ms-win-crt-runtime-l1-1-0.dll
 0001:00002b9a       _crt_atexit                0000000180003b9a f   ucrt:api-ms-win-crt-runtime-l1-1-0.dll
 0001:00002ba0       _cexit                     0000000180003ba0 f   ucrt:api-ms-win-crt-runtime-l1-1-0.dll
 0001:00002ba8       __acrt_initialize          0000000180003ba8 f   MSVCRT:ucrt_stubs.obj
 0001:00002ba8       __acrt_thread_attach       0000000180003ba8 f   MSVCRT:ucrt_stubs.obj
 0001:00002ba8       __acrt_thread_detach       0000000180003ba8 f   MSVCRT:ucrt_stubs.obj
 0001:00002ba8       __acrt_uninitialize        0000000180003ba8 f   MSVCRT:ucrt_stubs.obj
 0001:00002ba8       __acrt_uninitialize_critical 0000000180003ba8 f   MSVCRT:ucrt_stubs.obj
 0001:00002ba8       __scrt_stub_for_acrt_initialize 0000000180003ba8 f   MSVCRT:ucrt_stubs.obj
 0001:00002ba8       __scrt_stub_for_acrt_thread_attach 0000000180003ba8 f   MSVCRT:ucrt_stubs.obj
 0001:00002ba8       __scrt_stub_for_acrt_thread_detach 0000000180003ba8 f   MSVCRT:ucrt_stubs.obj
 0001:00002ba8       __scrt_stub_for_acrt_uninitialize 0000000180003ba8 f   MSVCRT:ucrt_stubs.obj
 0001:00002ba8       __scrt_stub_for_acrt_uninitialize_critical 0000000180003ba8 f   MSVCRT:ucrt_stubs.obj
 0001:00002ba8       __vcrt_initialize          0000000180003ba8 f   MSVCRT:ucrt_stubs.obj
 0001:00002ba8       __vcrt_thread_attach       0000000180003ba8 f   MSVCRT:ucrt_stubs.obj
 0001:00002ba8       __vcrt_thread_detach       0000000180003ba8 f   MSVCRT:ucrt_stubs.obj
 0001:00002ba8       __vcrt_uninitialize        0000000180003ba8 f   MSVCRT:ucrt_stubs.obj
 0001:00002ba8       __vcrt_uninitialize_critical 0000000180003ba8 f   MSVCRT:ucrt_stubs.obj
 0001:00002bac       __scrt_stub_for_is_c_termination_complete 0000000180003bac f   MSVCRT:ucrt_stubs.obj
 0001:00002bac       _is_c_termination_complete 0000000180003bac f   MSVCRT:ucrt_stubs.obj
 0001:00002bc0       _guard_dispatch_icall_nop  0000000180003bc0 f   MSVCRT:guard_dispatch.obj
 0001:00002be0       _guard_xfg_dispatch_icall_nop 0000000180003be0 f   MSVCRT:guard_xfg_dispatch.obj
 0002:00000000       __imp_RtlCaptureContext    0000000180004000     kernel32:KERNEL32.dll
 0002:00000008       __imp_RtlLookupFunctionEntry 0000000180004008     kernel32:KERNEL32.dll
 0002:00000010       __imp_RtlVirtualUnwind     0000000180004010     kernel32:KERNEL32.dll
 0002:00000018       __imp_UnhandledExceptionFilter 0000000180004018     kernel32:KERNEL32.dll
 0002:00000020       __imp_SetUnhandledExceptionFilter 0000000180004020     kernel32:KERNEL32.dll
 0002:00000028       __imp_GetCurrentProcess    0000000180004028     kernel32:KERNEL32.dll
 0002:00000030       __imp_TerminateProcess     0000000180004030     kernel32:KERNEL32.dll
 0002:00000038       __imp_IsProcessorFeaturePresent 0000000180004038     kernel32:KERNEL32.dll
 0002:00000040       __imp_CloseHandle          0000000180004040     kernel32:KERNEL32.dll
 0002:00000048       __imp_InitializeCriticalSectionAndSpinCount 0000000180004048     kernel32:KERNEL32.dll
 0002:00000050       __imp_DeleteCriticalSection 0000000180004050     kernel32:KERNEL32.dll
 0002:00000058       __imp_CreateEventW         0000000180004058     kernel32:KERNEL32.dll
 0002:00000060       __imp_GetModuleHandleW     0000000180004060     kernel32:KERNEL32.dll
 0002:00000068       __imp_GetProcAddress       0000000180004068     kernel32:KERNEL32.dll
 0002:00000070       __imp_IsDebuggerPresent    0000000180004070     kernel32:KERNEL32.dll
 0002:00000078       __imp_QueryPerformanceCounter 0000000180004078     kernel32:KERNEL32.dll
 0002:00000080       __imp_GetCurrentProcessId  0000000180004080     kernel32:KERNEL32.dll
 0002:00000088       __imp_GetCurrentThreadId   0000000180004088     kernel32:KERNEL32.dll
 0002:00000090       __imp_GetSystemTimeAsFileTime 0000000180004090     kernel32:KERNEL32.dll
 0002:00000098       __imp_DisableThreadLibraryCalls 0000000180004098     kernel32:KERNEL32.dll
 0002:000000a0       __imp_InitializeSListHead  00000001800040a0     kernel32:KERNEL32.dll
 0002:000000a8       \177KERNEL32_NULL_THUNK_DATA 00000001800040a8     kernel32:KERNEL32.dll
 0002:000000b0       __imp_memcpy               00000001800040b0     vcruntime:VCRUNTIME140.dll
 0002:000000b8       __imp_memset               00000001800040b8     vcruntime:VCRUNTIME140.dll
 0002:000000c0       __imp_strchr               00000001800040c0     vcruntime:VCRUNTIME140.dll
 0002:000000c8       __imp___C_specific_handler 00000001800040c8     vcruntime:VCRUNTIME140.dll
 0002:000000d0       __imp___std_type_info_destroy_list 00000001800040d0     vcruntime:VCRUNTIME140.dll
 0002:000000d8       \177VCRUNTIME140_NULL_THUNK_DATA 00000001800040d8     vcruntime:VCRUNTIME140.dll
 0002:000000e0       __imp__errno               00000001800040e0     ucrt:api-ms-win-crt-runtime-l1-1-0.dll
 0002:000000e8       __imp_exit                 00000001800040e8     ucrt:api-ms-win-crt-runtime-l1-1-0.dll
 0002:000000f0       __imp__cexit               00000001800040f0     ucrt:api-ms-win-crt-runtime-l1-1-0.dll
 0002:000000f8       __imp__crt_atexit          00000001800040f8     ucrt:api-ms-win-crt-runtime-l1-1-0.dll
 0002:00000100       __imp__execute_onexit_table 0000000180004100     ucrt:api-ms-win-crt-runtime-l1-1-0.dll
 0002:00000108       __imp__register_onexit_function 0000000180004108     ucrt:api-ms-win-crt-runtime-l1-1-0.dll
 0002:00000110       __imp__initialize_onexit_table 0000000180004110     ucrt:api-ms-win-crt-runtime-l1-1-0.dll
 0002:00000118       __imp__initialize_narrow_environment 0000000180004118     ucrt:api-ms-win-crt-runtime-l1-1-0.dll
 0002:00000120       __imp__configure_narrow_argv 0000000180004120     ucrt:api-ms-win-crt-runtime-l1-1-0.dll
 0002:00000128       __imp__seh_filter_dll      0000000180004128     ucrt:api-ms-win-crt-runtime-l1-1-0.dll
 0002:00000130       __imp__initterm_e          0000000180004130     ucrt:api-ms-win-crt-runtime-l1-1-0.dll
 0002:00000138       __imp__initterm            0000000180004138     ucrt:api-ms-win-crt-runtime-l1-1-0.dll
 0002:00000140       \177api-ms-win-crt-runtime-l1-1-0_NULL_THUNK_DATA 0000000180004140     ucrt:api-ms-win-crt-runtime-l1-1-0.dll
 0002:00000148       __imp___acrt_iob_func      0000000180004148     ucrt:api-ms-win-crt-stdio-l1-1-0.dll
 0002:00000150       __imp_fflush               0000000180004150     ucrt:api-ms-win-crt-stdio-l1-1-0.dll
 0002:00000158       __imp___stdio_common_vsprintf 0000000180004158     ucrt:api-ms-win-crt-stdio-l1-1-0.dll
 0002:00000160       __imp___stdio_common_vfprintf 0000000180004160     ucrt:api-ms-win-crt-stdio-l1-1-0.dll
 0002:00000168       \177api-ms-win-crt-stdio-l1-1-0_NULL_THUNK_DATA 0000000180004168     ucrt:api-ms-win-crt-stdio-l1-1-0.dll
 0002:00000170       __imp_strcmp               0000000180004170     ucrt:api-ms-win-crt-string-l1-1-0.dll
 0002:00000178       __imp__strdup              0000000180004178     ucrt:api-ms-win-crt-string-l1-1-0.dll
 0002:00000178       __imp_strdup               0000000180004178     ucrt:api-ms-win-crt-string-l1-1-0.dll
 0002:00000180       __imp_strlen               0000000180004180     ucrt:api-ms-win-crt-string-l1-1-0.dll
 0002:00000188       __imp_strncpy              0000000180004188     ucrt:api-ms-win-crt-string-l1-1-0.dll
 0002:00000190       \177api-ms-win-crt-string-l1-1-0_NULL_THUNK_DATA 0000000180004190     ucrt:api-ms-win-crt-string-l1-1-0.dll
 0002:00000198       __guard_check_icall_fptr   0000000180004198     MSVCRT:guard_support.obj
 0002:000001a0       __guard_xfg_check_icall_fptr 00000001800041a0     MSVCRT:guard_support.obj
 0002:000001a8       __guard_dispatch_icall_fptr 00000001800041a8     MSVCRT:guard_support.obj
 0002:000001b0       __guard_xfg_dispatch_icall_fptr 00000001800041b0     MSVCRT:guard_support.obj
 0002:000001b8       __guard_xfg_table_dispatch_icall_fptr 00000001800041b8     MSVCRT:guard_support.obj
 0002:000001c0       __castguard_check_failure_os_handled_fptr 00000001800041c0     MSVCRT:guard_support.obj
 0002:000001c8       __guard_memcpy_fptr        00000001800041c8     vcruntime:softmemtag.obj
 0002:000001d0       __xc_a                     00000001800041d0     MSVCRT:initializers.obj
 0002:000001d8       __xc_z                     00000001800041d8     MSVCRT:initializers.obj
 0002:000001e0       __xi_a                     00000001800041e0     MSVCRT:initializers.obj
 0002:000001f0       __xi_z                     00000001800041f0     MSVCRT:initializers.obj
 0002:000001f8       __xl_a                     00000001800041f8     MSVCRT:tlssup.obj
 0002:00000200       __xl_z                     0000000180004200     MSVCRT:tlssup.obj
 0002:00000208       __xp_a                     0000000180004208     MSVCRT:initializers.obj
 0002:00000210       __xp_z                     0000000180004210     MSVCRT:initializers.obj
 0002:00000218       __xt_a                     0000000180004218     MSVCRT:initializers.obj
 0002:00000220       __xt_z                     0000000180004220     MSVCRT:initializers.obj
 0002:00000230       ??_C@_06FALKBLGB@?$DMinit?$DO@ 0000000180004230     libbytecodes001.obj
 0002:00000240       g_refKindStr               0000000180004240     libbytecodes001.obj
 0002:000003f0       ??_C@_09BPLDFGCI@unknown_0@ 00000001800043f0     libbytecodes001.obj
 0002:00000400       ??_C@_0BL@FPNMECJD@JVMTI_HEAP_REFERENCE_CLASS@ 0000000180004400     libbytecodes001.obj
 0002:00000420       ??_C@_0BL@FKGKKLNM@JVMTI_HEAP_REFERENCE_FIELD@ 0000000180004420     libbytecodes001.obj
 0002:00000440       ??_C@_0CD@CAEHCFJF@JVMTI_HEAP_REFERENCE_ARRAY_ELEM@ 0000000180004440     libbytecodes001.obj
 0002:00000468       ??_C@_0CC@DNEBMCNK@JVMTI_HEAP_REFERENCE_CLASS_LOAD@ 0000000180004468     libbytecodes001.obj
 0002:00000490       ??_C@_0BN@CJMIPEBB@JVMTI_HEAP_REFERENCE_SIGNERS@ 0000000180004490     libbytecodes001.obj
 0002:000004b0       ??_C@_0CH@HBOIDPEB@JVMTI_HEAP_REFERENCE_PROTECTION@ 00000001800044b0     libbytecodes001.obj
 0002:000004d8       ??_C@_0BP@MDKGDGKL@JVMTI_HEAP_REFERENCE_INTERFACE@ 00000001800044d8     libbytecodes001.obj
 0002:000004f8       ??_C@_0CC@JJMIHNJH@JVMTI_HEAP_REFERENCE_STATIC_FIE@ 00000001800044f8     libbytecodes001.obj
 0002:00000520       ??_C@_0CD@IDHEEGID@JVMTI_HEAP_REFERENCE_CONSTANT_P@ 0000000180004520     libbytecodes001.obj
 0002:00000548       ??_C@_0CA@EFFCHNG@JVMTI_HEAP_REFERENCE_SUPERCLASS@ 0000000180004548     libbytecodes001.obj
 0002:00000568       ??_C@_0L@PCDFHGCJ@unknown_11@ 0000000180004568     libbytecodes001.obj
 0002:00000578       ??_C@_0L@NJBICFOK@unknown_12@ 0000000180004578     libbytecodes001.obj
 0002:00000588       ??_C@_0L@MAADBEKL@unknown_13@ 0000000180004588     libbytecodes001.obj
 0002:00000598       ??_C@_0L@IPECICGM@unknown_14@ 0000000180004598     libbytecodes001.obj
 0002:000005a8       ??_C@_0L@JGFJLDCN@unknown_15@ 00000001800045a8     libbytecodes001.obj
 0002:000005b8       ??_C@_0L@LNHEOAOO@unknown_16@ 00000001800045b8     libbytecodes001.obj
 0002:000005c8       ??_C@_0L@KEGPNBKP@unknown_17@ 00000001800045c8     libbytecodes001.obj
 0002:000005d8       ??_C@_0L@CDPHMNGA@unknown_18@ 00000001800045d8     libbytecodes001.obj
 0002:000005e8       ??_C@_0L@DKOMPMCB@unknown_19@ 00000001800045e8     libbytecodes001.obj
 0002:000005f8       ??_C@_0L@OJGIPJDB@unknown_20@ 00000001800045f8     libbytecodes001.obj
 0002:00000608       ??_C@_0CA@KAOFNDEM@JVMTI_HEAP_REFERENCE_JNI_GLOBAL@ 0000000180004608     libbytecodes001.obj
 0002:00000628       ??_C@_0CC@HPFAJBK@JVMTI_HEAP_REFERENCE_SYSTEM_CLA@ 0000000180004628     libbytecodes001.obj
 0002:00000650       ??_C@_0BN@FDEGFOHC@JVMTI_HEAP_REFERENCE_MONITOR@ 0000000180004650     libbytecodes001.obj
 0002:00000670       ??_C@_0CB@HKIBCMAJ@JVMTI_HEAP_REFERENCE_STACK_LOCA@ 0000000180004670     libbytecodes001.obj
 0002:00000698       ??_C@_0BP@EAACMMOE@JVMTI_HEAP_REFERENCE_JNI_LOCAL@ 0000000180004698     libbytecodes001.obj
 0002:000006b8       ??_C@_0BM@IJDEOGOE@JVMTI_HEAP_REFERENCE_THREAD@ 00000001800046b8     libbytecodes001.obj
 0002:000006d8       ??_C@_0BL@EDGPPKC@JVMTI_HEAP_REFERENCE_OTHER@ 00000001800046d8     libbytecodes001.obj
 0002:000006f4       ??_C@_04BCJPDBDA@Code@     00000001800046f4     libbytecodes001.obj
 0002:00000700       ??_C@_0BA@OCLMCFKC@LineNumberTable@ 0000000180004700     libbytecodes001.obj
 0002:00000710       ??_C@_0BD@CPAEPILC@LocalVariableTable@ 0000000180004710     libbytecodes001.obj
 0002:00000728       ??_C@_0BH@NMBDNHBD@LocalVariableTypeTable@ 0000000180004728     libbytecodes001.obj
 0002:00000740       ??_C@_0O@HIHEEDNJ@StackMapTable@ 0000000180004740     libbytecodes001.obj
 0002:00000750       ??_C@_03GAEACAIP@?$CI?$CJV@ 0000000180004750     libbytecodes001.obj
 0002:00000754       ??_C@_05MPEBBAAE@meth1@    0000000180004754     libbytecodes001.obj
 0002:0000075c       ??_C@_05OEGMEDMH@meth2@    000000018000475c     libbytecodes001.obj
 0002:00000764       ??_C@_05OLNBCKFJ@?$CII?$CJ?$FLF@ 0000000180004764     libbytecodes001.obj
 0002:00000770       ??_C@_0L@HCDIAMJG@?9?5?$CFs?0?5?$CFd?3?5@ 0000000180004770     libbytecodes001.obj
 0002:00000780       ??_C@_0JI@HLPECLFI@?$CD?5?4?4?4?6?$CD?5ERROR?3?5too?5many?5complai@ 0000000180004780     libbytecodes001.obj
 0002:00000820       ??_C@_0ED@JNEKCCOB@The?5following?5fake?5exception?5st@ 0000000180004820     libbytecodes001.obj
 0002:00000868       ??_C@_0CN@FCNMDFBH@nsk?4share?4Fake_Exception_for_RU@ 0000000180004868     libbytecodes001.obj
 0002:00000898       ??_C@_08PGFFNAEI@?$CI?$CFs?3?$CFd?$CJ?5@ 0000000180004898     libbytecodes001.obj
 0002:000008a8       ??_C@_0DP@IENMAEGI@s?2test?2hotspot?2jtreg?2vmTestbase@ 00000001800048a8     libbytecodes001.obj
 0002:000008e8       ??_C@_0BL@NDJLFFJB@?7at?5nsk_lvcomplain?$CI?$CFs?3?$CFd?$CJ?6@ 00000001800048e8     libbytecodes001.obj
 0002:00000908       ??_C@_0BC@JOOKAFKF@?$CD?5ERROR?3?5?$CFs?0?5?$CFd?3?5@ 0000000180004908     libbytecodes001.obj
 0002:00000920       ??_C@_09KJEAHMEH@?$CD?5ERROR?3?5@ 0000000180004920     libbytecodes001.obj
 0002:0000092c       ??_C@_02GPIOPFAK@?$DO?$DO@ 000000018000492c     libbytecodes001.obj
 0002:00000930       ??_C@_02FODMEDOG@?$DM?$DM@ 0000000180004930     libbytecodes001.obj
 0002:00000934       ??_C@_02DJGKEECL@?4?4@     0000000180004934     libbytecodes001.obj
 0002:00000938       ??_C@_0O@CJPGJOAF@?9?5?$CFs?0?5?$CFd?3?5?$CFs?5@ 0000000180004938     libbytecodes001.obj
 0002:00000948       ??_C@_0CB@IAKPDOIC@?$CD?5?5?5verified?5assertion?5is?5FALSE@ 0000000180004948     libbytecodes001.obj
 0002:00000970       ??_C@_0CO@LGONDEPD@stdout?3?5fflush?5failed?5?9?5err?$DN?$CFd?5@ 0000000180004970     libbytecodes001.obj
 0002:000009a0       ??_C@_0CO@KBGKJPBD@stderr?3?5fflush?5failed?5?9?5err?$DN?$CFd?5@ 00000001800049a0     libbytecodes001.obj
 0002:000009d0       ??_C@_0BB@JCNMKLLK@JVMTI_ERROR_NONE@ 00000001800049d0     libbytecodes001.obj
 0002:000009e8       ??_C@_0BL@LDIMKLPH@JVMTI_ERROR_INVALID_THREAD@ 00000001800049e8     libbytecodes001.obj
 0002:00000a08       ??_C@_0CB@PJFPAIKJ@JVMTI_ERROR_INVALID_THREAD_GROU@ 0000000180004a08     libbytecodes001.obj
 0002:00000a30       ??_C@_0BN@LLMKHMNF@JVMTI_ERROR_INVALID_PRIORITY@ 0000000180004a30     libbytecodes001.obj
 0002:00000a50       ??_C@_0CB@MBOFKAGB@JVMTI_ERROR_THREAD_NOT_SUSPENDE@ 0000000180004a50     libbytecodes001.obj
 0002:00000a78       ??_C@_0BN@FABOLPBI@JVMTI_ERROR_THREAD_SUSPENDED@ 0000000180004a78     libbytecodes001.obj
 0002:00000a98       ??_C@_0BN@FDGNOBJM@JVMTI_ERROR_THREAD_NOT_ALIVE@ 0000000180004a98     libbytecodes001.obj
 0002:00000ab8       ??_C@_0BL@GOBIFKNJ@JVMTI_ERROR_INVALID_OBJECT@ 0000000180004ab8     libbytecodes001.obj
 0002:00000ad8       ??_C@_0BK@FCMAJPPC@JVMTI_ERROR_INVALID_CLASS@ 0000000180004ad8     libbytecodes001.obj
 0002:00000af8       ??_C@_0BP@IKLLBKEB@JVMTI_ERROR_CLASS_NOT_PREPARED@ 0000000180004af8     libbytecodes001.obj
 0002:00000b18       ??_C@_0BN@KLPPLKG@JVMTI_ERROR_INVALID_METHODID@ 0000000180004b18     libbytecodes001.obj
 0002:00000b38       ??_C@_0BN@BCEKOKND@JVMTI_ERROR_INVALID_LOCATION@ 0000000180004b38     libbytecodes001.obj
 0002:00000b58       ??_C@_0BM@DFDGPME@JVMTI_ERROR_INVALID_FIELDID@ 0000000180004b58     libbytecodes001.obj
 0002:00000b78       ??_C@_0BL@NELIEPEC@JVMTI_ERROR_NO_MORE_FRAMES@ 0000000180004b78     libbytecodes001.obj
 0002:00000b98       ??_C@_0BJ@BDBECFDM@JVMTI_ERROR_OPAQUE_FRAME@ 0000000180004b98     libbytecodes001.obj
 0002:00000bb8       ??_C@_0BK@MIIFNLOB@JVMTI_ERROR_TYPE_MISMATCH@ 0000000180004bb8     libbytecodes001.obj
 0002:00000bd8       ??_C@_0BJ@HPCAOILC@JVMTI_ERROR_INVALID_SLOT@ 0000000180004bd8     libbytecodes001.obj
 0002:00000bf8       ??_C@_0BG@CHILOPNI@JVMTI_ERROR_DUPLICATE@ 0000000180004bf8     libbytecodes001.obj
 0002:00000c10       ??_C@_0BG@DIEMLHKM@JVMTI_ERROR_NOT_FOUND@ 0000000180004c10     libbytecodes001.obj
 0002:00000c28       ??_C@_0BM@NHMCKHOB@JVMTI_ERROR_INVALID_MONITOR@ 0000000180004c28     libbytecodes001.obj
 0002:00000c48       ??_C@_0BO@PPEDAJGL@JVMTI_ERROR_NOT_MONITOR_OWNER@ 0000000180004c48     libbytecodes001.obj
 0002:00000c68       ??_C@_0BG@FCAIPEID@JVMTI_ERROR_INTERRUPT@ 0000000180004c68     libbytecodes001.obj
 0002:00000c80       ??_C@_0CB@EGDBNKOI@JVMTI_ERROR_INVALID_CLASS_FORMA@ 0000000180004c80     libbytecodes001.obj
 0002:00000ca8       ??_C@_0CG@DGKOGIAL@JVMTI_ERROR_CIRCULAR_CLASS_DEFI@ 0000000180004ca8     libbytecodes001.obj
 0002:00000cd0       ??_C@_0BP@ICEALPKC@JVMTI_ERROR_FAILS_VERIFICATION@ 0000000180004cd0     libbytecodes001.obj
 0002:00000cf0       ??_C@_0DC@JDACLMIO@JVMTI_ERROR_UNSUPPORTED_REDEFIN@ 0000000180004cf0     libbytecodes001.obj
 0002:00000d28       ??_C@_0DE@GKDKNOMJ@JVMTI_ERROR_UNSUPPORTED_REDEFIN@ 0000000180004d28     libbytecodes001.obj
 0002:00000d60       ??_C@_0BO@LAFKIOG@JVMTI_ERROR_INVALID_TYPESTATE@ 0000000180004d60     libbytecodes001.obj
 0002:00000d80       ??_C@_0DH@INDGCLLB@JVMTI_ERROR_UNSUPPORTED_REDEFIN@ 0000000180004d80     libbytecodes001.obj
 0002:00000db8       ??_C@_0DE@NHEOMMGI@JVMTI_ERROR_UNSUPPORTED_REDEFIN@ 0000000180004db8     libbytecodes001.obj
 0002:00000df0       ??_C@_0CA@EKPNJOEP@JVMTI_ERROR_UNSUPPORTED_VERSION@ 0000000180004df0     libbytecodes001.obj
 0002:00000e10       ??_C@_0BN@OFFMAHHL@JVMTI_ERROR_NAMES_DONT_MATCH@ 0000000180004e10     libbytecodes001.obj
 0002:00000e30       ??_C@_0DN@HHBBLAKE@JVMTI_ERROR_UNSUPPORTED_REDEFIN@ 0000000180004e30     libbytecodes001.obj
 0002:00000e70       ??_C@_0DO@HMBGBGNA@JVMTI_ERROR_UNSUPPORTED_REDEFIN@ 0000000180004e70     libbytecodes001.obj
 0002:00000eb0       ??_C@_0BP@PBECGKHJ@JVMTI_ERROR_UNMODIFIABLE_CLASS@ 0000000180004eb0     libbytecodes001.obj
 0002:00000ed0       ??_C@_0BK@CANILEHF@JVMTI_ERROR_NOT_AVAILABLE@ 0000000180004ed0     libbytecodes001.obj
 0002:00000ef0       ??_C@_0CE@INJKMEFK@JVMTI_ERROR_MUST_POSSESS_CAPABI@ 0000000180004ef0     libbytecodes001.obj
 0002:00000f18       ??_C@_0BJ@LBFPFPDM@JVMTI_ERROR_NULL_POINTER@ 0000000180004f18     libbytecodes001.obj
 0002:00000f38       ??_C@_0BP@CHJPNNEM@JVMTI_ERROR_ABSENT_INFORMATION@ 0000000180004f38     libbytecodes001.obj
 0002:00000f58       ??_C@_0BP@OMFMNLC@JVMTI_ERROR_INVALID_EVENT_TYPE@ 0000000180004f58     libbytecodes001.obj
 0002:00000f78       ??_C@_0BN@BIBNPHHO@JVMTI_ERROR_ILLEGAL_ARGUMENT@ 0000000180004f78     libbytecodes001.obj
 0002:00000f98       ??_C@_0BK@KKNDHDCE@JVMTI_ERROR_NATIVE_METHOD@ 0000000180004f98     libbytecodes001.obj
 0002:00000fb8       ??_C@_0BK@PMKCFHAE@JVMTI_ERROR_OUT_OF_MEMORY@ 0000000180004fb8     libbytecodes001.obj
 0002:00000fd8       ??_C@_0BK@NNJBDMNB@JVMTI_ERROR_ACCESS_DENIED@ 0000000180004fd8     libbytecodes001.obj
 0002:00000ff8       ??_C@_0BI@GHECLMNC@JVMTI_ERROR_WRONG_PHASE@ 0000000180004ff8     libbytecodes001.obj
 0002:00001010       ??_C@_0BF@OLIHJOII@JVMTI_ERROR_INTERNAL@ 0000000180005010     libbytecodes001.obj
 0002:00001028       ??_C@_0BO@EOHGKJHI@JVMTI_ERROR_UNATTACHED_THREAD@ 0000000180005028     libbytecodes001.obj
 0002:00001048       ??_C@_0CA@LKHFDACL@JVMTI_ERROR_INVALID_ENVIRONMENT@ 0000000180005048     libbytecodes001.obj
 0002:00001068       ??_C@_0BA@MMFHLOKK@?$DMunknown?5error?$DO@ 0000000180005068     libbytecodes001.obj
 0002:00001078       ??_C@_0CF@CBHOKDB@throwable?5?$DN?5jni?9?$DOExceptionOccur@ 0000000180005078     libbytecodes001.obj
 0002:000010a0       ??_C@_03OFAPEBGM@?$CFs?6@  00000001800050a0     libbytecodes001.obj
 0002:000010a8       ??_C@_0DM@LPIGEGNJ@s?2test?2hotspot?2jtreg?2vmTestbase@ 00000001800050a8     libbytecodes001.obj
 0002:000010e8       ??_C@_0CC@NFCNPEPK@Exception?5in?5JNI?5call?5?$CIcleared?$CJ@ 00000001800050e8     libbytecodes001.obj
 0002:00001110       ??_C@_0BJ@IBAKFIKF@jni?9?$DOExceptionDescribe?$CI?$CJ@ 0000000180005110     libbytecodes001.obj
 0002:00001130       ??_C@_0BG@GGKALKMH@jni?9?$DOExceptionClear?$CI?$CJ@ 0000000180005130     libbytecodes001.obj
 0002:00001148       ??_C@_0CF@JMGFGJLJ@?$CD?5?5?5verified?5JNI?5assertion?5is?5F@ 0000000180005148     libbytecodes001.obj
 0002:00001170       ??_C@_0CB@MLNJNCLJ@?5?5jvmti?5error?3?5code?$DN?$CFd?0?5name?$DN?$CFs@ 0000000180005170     libbytecodes001.obj
 0002:00001198       ??_C@_0CD@OHBGDKMK@?$CD?5?5?5jvmti?5error?3?5code?$DN?$CFd?0?5name?$DN@ 0000000180005198     libbytecodes001.obj
 0002:000011c0       ??_C@_0CG@JNNCGPHB@?$CD?5?5?5error?5expected?3?5code?$DN?$CFd?0?5na@ 00000001800051c0     libbytecodes001.obj
 0002:000011f0       ??_C@_0EB@IMGKPCGE@?$CIstr_obj?5?$DN?5jni?9?$DONewStringUTF?$CIco@ 00000001800051f0     libbytecodes001.obj
 0002:00001240       ??_C@_0EA@HFOGGBCC@s?2test?2hotspot?2jtreg?2vmTestbase@ 0000000180005240     libbytecodes001.obj
 0002:00001280       ??_C@_05KKCIMGE@error@     0000000180005280     libbytecodes001.obj
 0002:00001290       ??_C@_0EA@PNBCDMOA@s?2test?2hotspot?2jtreg?2vmTestbase@ 0000000180005290     libbytecodes001.obj
 0002:000012d0       ??_C@_0DI@ILAHDLMP@?$CI?$CKagentThreadProc?$CJ?$CIjvmti_env?0?5a@ 00000001800052d0     libbytecodes001.obj
 0002:00001308       ??_C@_0BD@KDBALNLB@JVMTI?5agent?5thread@ 0000000180005308     libbytecodes001.obj
 0002:00001320       ??_C@_0BB@NOKBFPFO@java?1lang?1Thread@ 0000000180005320     libbytecodes001.obj
 0002:00001338       ??_C@_0BG@IKDDPPGD@?$CILjava?1lang?1String?$DL?$CJV@ 0000000180005338     libbytecodes001.obj
 0002:00001350       ??_C@_0EB@IFJBFEKC@?$CIthreadClass?5?$DN?5jni_env?9?$DOFindCla@ 0000000180005350     libbytecodes001.obj
 0002:000013a0       ??_C@_0GF@FGFIBKKL@?$CIthreadCtor?5?$DN?5jni_env?9?$DOGetMetho@ 00000001800053a0     libbytecodes001.obj
 0002:00001408       ??_C@_0DN@NCPDJLOG@?$CIthreadName?5?$DN?5jni_env?9?$DONewStrin@ 0000000180005408     libbytecodes001.obj
 0002:00001450       ??_C@_0FE@PFKODBGC@?$CIthreadObject?5?$DN?5jni_env?9?$DONewObj@ 0000000180005450     libbytecodes001.obj
 0002:000014b0       ??_C@_0ED@HOBAHHJI@?$CIthreadGlobalRef?5?$DN?5jni_env?9?$DONew@ 00000001800054b0     libbytecodes001.obj
 0002:00001500       ??_C@_0FN@HNJJAHFC@jvmti_env?9?$DORunAgentThread?$CIagent@ 0000000180005500     libbytecodes001.obj
 0002:00001560       ??_C@_0EA@MOJDNKDF@Debuggee?5status?5sync?5aborted?5be@ 0000000180005560     libbytecodes001.obj
 0002:000015a0       ??_C@_0EA@EEOEJAEN@status?5?$DN?5syncDebuggeeStatus?$CIjni@ 00000001800055a0     libbytecodes001.obj
 0002:000015e0       ??_C@_0BL@JBCFNBMB@nsk_jvmti_resetAgentData?$CI?$CJ@ 00000001800055e0     libbytecodes001.obj
 0002:00001600       ??_C@_0EL@LPBEELIP@s?2test?2hotspot?2jtreg?2vmTestbase@ 0000000180005600     libbytecodes001.obj
 0002:00001650       ??_C@_0CK@JDAMFDMJ@jvmti?9?$DOSetTag?$CIo?0?5tag?$CJ?5?$DN?$DN?5JVMTI_@ 0000000180005650     libbytecodes001.obj
 0002:00001680       ??_C@_0CC@DAMNHKNI@Can?8t?5set?5tag?5?$CFli?5for?5object?5?$CFl@ 0000000180005680     libbytecodes001.obj
 0002:000016a8       ??_C@_0DL@HAJPNKEF@jvmti?9?$DOGetObjectHashCode?$CIo?0?5?$CGha@ 00000001800056a8     libbytecodes001.obj
 0002:000016e8       ??_C@_0BL@JFPIEOBF@Can?8t?5get?5hash?5object?5?$CFlx?6@ 00000001800056e8     libbytecodes001.obj
 0002:00001708       ??_C@_0BG@DICPHBKN@setTag?3?5?$CF08x?5?$DM?9?5?$CF?53li@ 0000000180005708     libbytecodes001.obj
 0002:00001720       ??_C@_0DH@FCEEBDMJ@?$CIs?5?$DN?5jni?9?$DOGetStringUTFChars?$CIsIn@ 0000000180005720     libbytecodes001.obj
 0002:00001758       ??_C@_0BJ@OKKGHDCN@Can?8t?5get?5string?5at?5?$CF?$CDp?6@ 0000000180005758     libbytecodes001.obj
 0002:00001778       ??_C@_0BP@EKFLGGFJ@Can?8t?5get?5string?5at?5?$CF?$CDp?3?5null?6@ 0000000180005778     libbytecodes001.obj
 0002:00001798       ??_C@_06ICODBHCL@?5?1?1?5?$CFs@ 0000000180005798     libbytecodes001.obj
 0002:000017a0       ??_C@_0DB@KGFPLEGO@?$CIr?5?$DN?5jvmti?9?$DOGetTag?$CIo?0?5?$CGtag?$CJ?$CJ?5?$DN?$DN@ 00000001800057a0     libbytecodes001.obj
 0002:000017d8       ??_C@_0CO@PDAGBCGJ@Can?8t?5GetTag?5for?5object?5?$CFlx?4?5Re@ 00000001800057d8     libbytecodes001.obj
 0002:00001808       ??_C@_0CH@HPEODOHC@TEST_BUG?3?5Max?4?5number?5of?5refs?5r@ 0000000180005808     libbytecodes001.obj
 0002:00001830       ??_C@_0DI@PHFCABIM@?$CIr?5?$DN?5jvmti?9?$DOGetTag?$CIfrom?0?5?$CGtagFr@ 0000000180005830     libbytecodes001.obj
 0002:00001868       ??_C@_0DI@MDEGFNKD@TEST_BUG?3?5Can?8t?5GetTag?5for?5obje@ 0000000180005868     libbytecodes001.obj
 0002:000018a0       ??_C@_0DE@MLELJAHM@?$CIr?5?$DN?5jvmti?9?$DOGetTag?$CIto?0?5?$CGtagTo?$CJ?$CJ@ 00000001800058a0     libbytecodes001.obj
 0002:000018d8       ??_C@_09OPJEJKBL@printdump@ 00000001800058d8     libbytecodes001.obj
 0002:000018e8       ??_C@_0CJ@KCDEKOCJ@Wrong?5result?5of?5a?5valid?5call?5to@ 00000001800058e8     libbytecodes001.obj
 0002:00001918       ??_C@_0CN@BCCBOHCH@?$CIGetCapabilities?$CJ?5unexpected?5er@ 0000000180005918     libbytecodes001.obj
 0002:00001948       ??_C@_0DG@LAJPGIIE@?$CIGetPotentialCapabilities?$CJ?5unex@ 0000000180005948     libbytecodes001.obj
 0002:00001980       ??_C@_0CN@LKPEOJPO@?$CIAddCapabilities?$CJ?5unexpected?5er@ 0000000180005980     libbytecodes001.obj
 0002:000019b0       ??_C@_0CK@EFOMNEB@Warning?3?5GetBytecodes?5is?5not?5im@ 00000001800059b0     libbytecodes001.obj
 0002:000019e0       ??_C@_0CH@CDOJMNAO@JVMTI?5client?5was?5not?5properly?5l@ 00000001800059e0     libbytecodes001.obj
 0002:00001a08       ??_C@_0BP@DOJMFIJG@?$CC?$CFs?$CFs?$CC?3?5cannot?5get?5method?5ID?$CB?6@ 0000000180005a08     libbytecodes001.obj
 0002:00001a28       ??_C@_0BG@NOGMCOAI@?$DO?$DO?$DO?5?$CC?$CFs?$CFs?$CC?5check?5?4?4?4?6@ 0000000180005a28     libbytecodes001.obj
 0002:00001a40       ??_C@_0CN@BCJOCBI@?$CIGetBytecodes?$CD?$CFs?$CJ?5unexpected?5er@ 0000000180005a40     libbytecodes001.obj
 0002:00001a70       ??_C@_0DD@HPFLMPFK@?$CC?$CFs?$CFs?$CC?3?5byte?5codes?5count?5expect@ 0000000180005a70     libbytecodes001.obj
 0002:00001aa8       ??_C@_0DA@IFMIENMI@?$CC?$CFs?$CFs?$CC?3?5?$FL?$CFd?$FN?5byte?5expected?3?50x?$CF@ 0000000180005aa8     libbytecodes001.obj
 0002:00001af0       ??_C@_1EC@JIJBPKFM@?$AAa?$AAp?$AAi?$AA?9?$AAm?$AAs?$AA?9?$AAw?$AAi?$AAn?$AA?9?$AAc?$AAo?$AAr?$AAe@ 0000000180005af0     MSVCRT:thread_safe_statics.obj
 0002:00001b38       ??_C@_1BK@MGMFAEKH@?$AAk?$AAe?$AAr?$AAn?$AAe?$AAl?$AA3?$AA2?$AA?4?$AAd?$AAl?$AAl@ 0000000180005b38     MSVCRT:thread_safe_statics.obj
 0002:00001b58       ??_C@_0BJ@JEBJOJFJ@SleepConditionVariableCS@ 0000000180005b58     MSVCRT:thread_safe_statics.obj
 0002:00001b78       ??_C@_0BJ@PGPPEPCC@WakeAllConditionVariable@ 0000000180005b78     MSVCRT:thread_safe_statics.obj
 0002:00001b98       _pDefaultRawDllMain        0000000180005b98     MSVCRT:dll_dllmain.obj
 0002:00001b98       _pRawDllMain               0000000180005b98     MSVCRT:dll_dllmain.obj
 0002:00001ba0       __xmm@ffffffffffffffffffffffffffffffff 0000000180005ba0     MSVCRT:utility.obj
 0002:00001bb0       _load_config_used          0000000180005bb0     MSVCRT:loadcfg.obj
 0002:00001d80       _tls_used                  0000000180005d80     MSVCRT:tlssup.obj
 0002:00001da8       __volatile_metadata        0000000180005da8     <linker-defined>
 0002:00002178       __rtc_iaa                  0000000180006178     MSVCRT:initsect.obj
 0002:00002180       __rtc_izz                  0000000180006180     MSVCRT:initsect.obj
 0002:00002188       __rtc_taa                  0000000180006188     MSVCRT:initsect.obj
 0002:00002190       __rtc_tzz                  0000000180006190     MSVCRT:initsect.obj
 0002:00002198       _tls_start                 0000000180006198     MSVCRT:tlssup.obj
 0002:0000219c       _Init_thread_epoch         000000018000619c     MSVCRT:thread_safe_statics.obj
 0002:000021a0       _tls_end                   00000001800061a0     MSVCRT:tlssup.obj
 0002:00002830       __IMPORT_DESCRIPTOR_KERNEL32 0000000180006830     kernel32:KERNEL32.dll
 0002:00002844       __IMPORT_DESCRIPTOR_VCRUNTIME140 0000000180006844     vcruntime:VCRUNTIME140.dll
 0002:00002858       __IMPORT_DESCRIPTOR_api-ms-win-crt-runtime-l1-1-0 0000000180006858     ucrt:api-ms-win-crt-runtime-l1-1-0.dll
 0002:0000286c       __IMPORT_DESCRIPTOR_api-ms-win-crt-stdio-l1-1-0 000000018000686c     ucrt:api-ms-win-crt-stdio-l1-1-0.dll
 0002:00002880       __IMPORT_DESCRIPTOR_api-ms-win-crt-string-l1-1-0 0000000180006880     ucrt:api-ms-win-crt-string-l1-1-0.dll
 0002:00002894       __NULL_IMPORT_DESCRIPTOR   0000000180006894     kernel32:KERNEL32.dll
 0003:000000a0       _Init_global_epoch         00000001800070a0     MSVCRT:thread_safe_statics.obj
 0003:000000b0       __security_cookie          00000001800070b0     MSVCRT:gs_cookie.obj
 0003:000000b8       __security_cookie_complement 00000001800070b8     MSVCRT:gs_cookie.obj
 0003:000000c0       __scrt_native_dllmain_reason 00000001800070c0     MSVCRT:utility.obj
 0003:000000c8       __isa_available            00000001800070c8     MSVCRT:cpu_disp.obj
 0003:000000cc       __isa_enabled              00000001800070cc     MSVCRT:cpu_disp.obj
 0003:000000d0       __memset_fast_string_threshold 00000001800070d0     MSVCRT:cpu_disp.obj
 0003:000000d8       __memset_nt_threshold      00000001800070d8     MSVCRT:cpu_disp.obj
 0003:000000e0       __scrt_ucrt_dll_is_in_use  00000001800070e0     MSVCRT:ucrt_stubs.obj
 0003:000000f0       g_wrongHeapCallbacks       00000001800070f0     libbytecodes001.obj
 0003:00000170       g_szTagInfo                0000000180007170     libbytecodes001.obj
 0003:000020b0       g_tagFlags                 00000001800090b0     libbytecodes001.obj
 0003:00002498       g_refsToVerifyCnt          0000000180009498     libbytecodes001.obj
 0003:0000249c       g_fakeUserData             000000018000949c     libbytecodes001.obj
 0003:000024a0       g_tagVisitCount            00000001800094a0     libbytecodes001.obj
 0003:00003440       g_refsToVerify             000000018000a440     libbytecodes001.obj
 0003:0001ab40       g_userDataError            0000000180021b40     libbytecodes001.obj
 0003:0001acf0       ?_OptionsStorage@?1??__local_stdio_printf_options@@9@4_KA 0000000180021cf0     libbytecodes001.obj
 0003:0001b2b8       _tls_index                 00000001800222b8     MSVCRT:tlssup.obj
 0003:0001b2c0       __scrt_current_native_startup_state 00000001800222c0     MSVCRT:utility.obj
 0003:0001b2c8       __scrt_native_startup_lock 00000001800222c8     MSVCRT:utility.obj
 0003:0001b308       __scrt_debugger_hook_flag  0000000180022308     MSVCRT:utility_desktop.obj
 0003:0001b310       ?__type_info_root_node@@3U__type_info_node@@A 0000000180022310     MSVCRT:tncleanup.obj
 0003:0001b320       ?_OptionsStorage@?1??__local_stdio_scanf_options@@9@4_KA 0000000180022320     MSVCRT:default_local_stdio_options.obj
 0003:0001b328       __favor                    0000000180022328     MSVCRT:cpu_disp.obj
 0003:0001b330       __dyn_tls_init_callback    0000000180022330     <common>

 entry point at        0001:000022d0

 Static symbols

 0000:fffdb000       .debug$S                   0000000180000000     bytecodes001.exp
 0000:fffdb000       .debug$S                   0000000180000000     vcruntime:VCRUNTIME140.dll
 0000:fffdb000       .debug$S                   0000000180000000     vcruntime:VCRUNTIME140.dll
 0000:fffdb000       .debug$S                   0000000180000000     vcruntime:VCRUNTIME140.dll
 0000:fffdb000       .debug$S                   0000000180000000     vcruntime:VCRUNTIME140.dll
 0000:fffdb000       .debug$S                   0000000180000000     vcruntime:VCRUNTIME140.dll
 0000:fffdb000       .debug$S                   0000000180000000     vcruntime:VCRUNTIME140.dll
 0000:fffdb000       .debug$S                   0000000180000000     vcruntime:VCRUNTIME140.dll
 0000:fffdb000       .debug$S                   0000000180000000     ucrt:api-ms-win-crt-convert-l1-1-0.dll
 0002:ffffc000       .idata$6                   0000000180000000     ucrt:api-ms-win-crt-convert-l1-1-0.dll
 0000:fffdb000       .debug$S                   0000000180000000     ucrt:api-ms-win-crt-heap-l1-1-0.dll
 0000:fffdb000       .debug$S                   0000000180000000     ucrt:api-ms-win-crt-heap-l1-1-0.dll
 0000:fffdb000       .debug$S                   0000000180000000     ucrt:api-ms-win-crt-heap-l1-1-0.dll
 0000:fffdb000       .debug$S                   0000000180000000     ucrt:api-ms-win-crt-heap-l1-1-0.dll
 0002:ffffc000       .idata$6                   0000000180000000     ucrt:api-ms-win-crt-heap-l1-1-0.dll
 0000:fffdb000       .debug$S                   0000000180000000     ucrt:api-ms-win-crt-runtime-l1-1-0.dll
 0000:fffdb000       .debug$S                   0000000180000000     ucrt:api-ms-win-crt-runtime-l1-1-0.dll
 0000:fffdb000       .debug$S                   0000000180000000     ucrt:api-ms-win-crt-runtime-l1-1-0.dll
 0000:fffdb000       .debug$S                   0000000180000000     ucrt:api-ms-win-crt-runtime-l1-1-0.dll
 0000:fffdb000       .debug$S                   0000000180000000     ucrt:api-ms-win-crt-runtime-l1-1-0.dll
 0000:fffdb000       .debug$S                   0000000180000000     ucrt:api-ms-win-crt-runtime-l1-1-0.dll
 0000:fffdb000       .debug$S                   0000000180000000     ucrt:api-ms-win-crt-runtime-l1-1-0.dll
 0000:fffdb000       .debug$S                   0000000180000000     ucrt:api-ms-win-crt-runtime-l1-1-0.dll
 0000:fffdb000       .debug$S                   0000000180000000     ucrt:api-ms-win-crt-runtime-l1-1-0.dll
 0000:fffdb000       .debug$S                   0000000180000000     ucrt:api-ms-win-crt-runtime-l1-1-0.dll
 0000:fffdb000       .debug$S                   0000000180000000     ucrt:api-ms-win-crt-runtime-l1-1-0.dll
 0000:fffdb000       .debug$S                   0000000180000000     ucrt:api-ms-win-crt-runtime-l1-1-0.dll
 0000:fffdb000       .debug$S                   0000000180000000     ucrt:api-ms-win-crt-runtime-l1-1-0.dll
 0000:fffdb000       .debug$S                   0000000180000000     ucrt:api-ms-win-crt-runtime-l1-1-0.dll
 0000:fffdb000       .debug$S                   0000000180000000     ucrt:api-ms-win-crt-runtime-l1-1-0.dll
 0000:fffdb000       .debug$S                   0000000180000000     ucrt:api-ms-win-crt-runtime-l1-1-0.dll
 0000:fffdb000       .debug$S                   0000000180000000     ucrt:api-ms-win-crt-stdio-l1-1-0.dll
 0000:fffdb000       .debug$S                   0000000180000000     ucrt:api-ms-win-crt-stdio-l1-1-0.dll
 0000:fffdb000       .debug$S                   0000000180000000     ucrt:api-ms-win-crt-stdio-l1-1-0.dll
 0000:fffdb000       .debug$S                   0000000180000000     ucrt:api-ms-win-crt-stdio-l1-1-0.dll
 0000:fffdb000       .debug$S                   0000000180000000     ucrt:api-ms-win-crt-stdio-l1-1-0.dll
 0000:fffdb000       .debug$S                   0000000180000000     ucrt:api-ms-win-crt-stdio-l1-1-0.dll
 0000:fffdb000       .debug$S                   0000000180000000     ucrt:api-ms-win-crt-stdio-l1-1-0.dll
 0000:fffdb000       .debug$S                   0000000180000000     ucrt:api-ms-win-crt-stdio-l1-1-0.dll
 0000:fffdb000       .debug$S                   0000000180000000     ucrt:api-ms-win-crt-stdio-l1-1-0.dll
 0000:fffdb000       .debug$S                   0000000180000000     ucrt:api-ms-win-crt-stdio-l1-1-0.dll
 0000:fffdb000       .debug$S                   0000000180000000     ucrt:api-ms-win-crt-string-l1-1-0.dll
 0000:fffdb000       .debug$S                   0000000180000000     ucrt:api-ms-win-crt-string-l1-1-0.dll
 0000:fffdb000       .debug$S                   0000000180000000     ucrt:api-ms-win-crt-string-l1-1-0.dll
 0000:fffdb000       .debug$S                   0000000180000000     ucrt:api-ms-win-crt-string-l1-1-0.dll
 0000:fffdb000       .debug$S                   0000000180000000     ucrt:api-ms-win-crt-string-l1-1-0.dll
 0000:fffdb000       .debug$S                   0000000180000000     ucrt:api-ms-win-crt-string-l1-1-0.dll
 0000:fffdb000       .debug$S                   0000000180000000     ucrt:api-ms-win-crt-string-l1-1-0.dll
 0000:fffdb000       .debug$S                   0000000180000000     ucrt:api-ms-win-crt-string-l1-1-0.dll
 0000:fffdb000       .debug$S                   0000000180000000     kernel32:KERNEL32.dll
 0000:fffdb000       .debug$S                   0000000180000000     kernel32:KERNEL32.dll
 0000:fffdb000       .debug$S                   0000000180000000     kernel32:KERNEL32.dll
 0000:fffdb000       .debug$S                   0000000180000000     kernel32:KERNEL32.dll
 0000:fffdb000       .debug$S                   0000000180000000     kernel32:KERNEL32.dll
 0000:fffdb000       .debug$S                   0000000180000000     kernel32:KERNEL32.dll
 0000:fffdb000       .debug$S                   0000000180000000     kernel32:KERNEL32.dll
 0000:fffdb000       .debug$S                   0000000180000000     kernel32:KERNEL32.dll
 0000:fffdb000       .debug$S                   0000000180000000     kernel32:KERNEL32.dll
 0000:fffdb000       .debug$S                   0000000180000000     kernel32:KERNEL32.dll
 0000:fffdb000       .debug$S                   0000000180000000     kernel32:KERNEL32.dll
 0000:fffdb000       .debug$S                   0000000180000000     kernel32:KERNEL32.dll
 0000:fffdb000       .debug$S                   0000000180000000     kernel32:KERNEL32.dll
 0000:fffdb000       .debug$S                   0000000180000000     kernel32:KERNEL32.dll
 0000:fffdb000       .debug$S                   0000000180000000     kernel32:KERNEL32.dll
 0000:fffdb000       .debug$S                   0000000180000000     kernel32:KERNEL32.dll
 0000:fffdb000       .debug$S                   0000000180000000     kernel32:KERNEL32.dll
 0000:fffdb000       .debug$S                   0000000180000000     kernel32:KERNEL32.dll
 0000:fffdb000       .debug$S                   0000000180000000     kernel32:KERNEL32.dll
 0000:fffdb000       .debug$S                   0000000180000000     kernel32:KERNEL32.dll
 0000:fffdb000       .debug$S                   0000000180000000     kernel32:KERNEL32.dll
 0000:fffdb000       .debug$S                   0000000180000000     kernel32:KERNEL32.dll
 0000:fffdb000       .debug$S                   0000000180000000     kernel32:KERNEL32.dll
 0000:fffdb000       .debug$S                   0000000180000000     kernel32:KERNEL32.dll
 0000:fffdb000       .debug$S                   0000000180000000     kernel32:KERNEL32.dll
 0000:fffdb000       .debug$S                   0000000180000000     kernel32:KERNEL32.dll
 0000:fffdb000       .debug$S                   0000000180000000     kernel32:KERNEL32.dll
 0000:fffdb000       .debug$S                   0000000180000000     kernel32:KERNEL32.dll
 0001:00000dcc       addRefToVerify             0000000180001dcc f   libbytecodes001.obj
 0001:00000e40       agentThreadWrapper         0000000180001e40 f   libbytecodes001.obj
 0001:000011bc       file_basename              00000001800021bc f   libbytecodes001.obj
 0001:000017e4       startAgentThreadWrapper    00000001800027e4 f   libbytecodes001.obj
 0001:00001b10       syncDebuggeeStatus         0000000180002b10 f   libbytecodes001.obj
 0001:00001d98       capture_previous_context   0000000180002d98 f   MSVCRT:gs_report.obj
 0001:00001e0c       ?__scrt_initialize_thread_safe_statics@@YAHXZ 0000000180002e0c f   MSVCRT:thread_safe_statics.obj
 0001:00001edc       ?__scrt_uninitialize_thread_safe_statics@@YAXXZ 0000000180002edc f   MSVCRT:thread_safe_statics.obj
 0001:00001f80       $$000000                   0000000180002f80     MSVCRT:amdsecgs.obj
 0001:00001fb0       ?dllmain_crt_dispatch@@YAHQEAUHINSTANCE__@@KQEAX@Z 0000000180002fb0 f   MSVCRT:dll_dllmain.obj
 0001:00002000       ?dllmain_crt_process_attach@@YAHQEAUHINSTANCE__@@QEAX@Z 0000000180003000 f   MSVCRT:dll_dllmain.obj
 0001:00002118       ?dllmain_crt_process_detach@@YAH_N@Z 0000000180003118 f   MSVCRT:dll_dllmain.obj
 0001:0000219c       ?dllmain_dispatch@@YAHQEAUHINSTANCE__@@KQEAX@Z 000000018000319c f   MSVCRT:dll_dllmain.obj
 0001:00002bb0       $$000000                   0000000180003bb0     MSVCRT:guard_dispatch.obj
 0001:00002bd0       $$000000                   0000000180003bd0     MSVCRT:guard_xfg_dispatch.obj
 0001:00002be6       ?fin$0@?0??dllmain_crt_process_attach@@YAHQEAUHINSTANCE__@@QEAX@Z@4HA 0000000180003be6 f   MSVCRT:dll_dllmain.obj
 0001:00002bfd       ?fin$0@?0??dllmain_crt_process_detach@@YAH_N@Z@4HA 0000000180003bfd f   MSVCRT:dll_dllmain.obj
 0001:00002c16       ?fin$1@?0??dllmain_crt_process_detach@@YAH_N@Z@4HA 0000000180003c16 f   MSVCRT:dll_dllmain.obj
 0001:00002c2a       ?filt$0@?0??dllmain_dispatch@@YAHQEAUHINSTANCE__@@KQEAX@Z@4HA 0000000180003c2a f   MSVCRT:dll_dllmain.obj
 0001:00002c60       __scrt_is_nonwritable_in_current_image$filt$0 0000000180003c60 f   MSVCRT:utility.obj
 0002:000001e8       ?__scrt_initialize_tss_var@@3P6AHXZEA 00000001800041e8     MSVCRT:thread_safe_statics.obj
 0002:00000320       ?opcLengths@@3QBEB         0000000180004320     libbytecodes001.obj
 0002:00001ad8       GS_ExceptionPointers       0000000180005ad8     MSVCRT:gs_report.obj
 0002:000021a8       $unwind$fprintf            00000001800061a8     libbytecodes001.obj
 0002:000021b4       $unwind$printf             00000001800061b4     libbytecodes001.obj
 0002:000021c0       $unwind$?NewObject@JNIEnv_@@QEAAPEAV_jobject@@PEAV_jclass@@PEAU_jmethodID@@ZZ 00000001800061c0     libbytecodes001.obj
 0002:000021c0       $unwind$nsk_lcomplain      00000001800061c0     libbytecodes001.obj
 0002:000021c0       $unwind$nsk_ldisplay       00000001800061c0     libbytecodes001.obj
 0002:000021c8       $unwind$Java_nsk_jvmti_GetBytecodes_bytecodes001_check 00000001800061c8     libbytecodes001.obj
 0002:000021c8       $unwind$nsk_lvdisplay      00000001800061c8     libbytecodes001.obj
 0002:000021c8       $unwind$_RTC_Initialize    00000001800061c8     MSVCRT:initsect.obj
 0002:000021c8       $unwind$_RTC_Terminate     00000001800061c8     MSVCRT:initsect.obj
 0002:000021c8       $unwind$?__scrt_initialize_thread_safe_statics@@YAHXZ 00000001800061c8     MSVCRT:thread_safe_statics.obj
 0002:000021d4       $unwind$nsk_lvcomplain     00000001800061d4     libbytecodes001.obj
 0002:000021ec       $unwind$nsk_ltrace         00000001800061ec     libbytecodes001.obj
 0002:000021ec       $unwind$__report_gsfailure 00000001800061ec     MSVCRT:gs_report.obj
 0002:000021f4       $unwind$Agent_Initialize   00000001800061f4     libbytecodes001.obj
 0002:000021f4       $unwind$nsk_lvtrace        00000001800061f4     libbytecodes001.obj
 0002:000021f4       $unwind$__raise_securityfailure 00000001800061f4     MSVCRT:gs_report.obj
 0002:000021f4       $unwind$__scrt_initialize_crt 00000001800061f4     MSVCRT:utility.obj
 0002:000021f4       $unwind$__scrt_initialize_onexit_tables 00000001800061f4     MSVCRT:utility.obj
 0002:000021f4       $unwind$__scrt_release_startup_lock 00000001800061f4     MSVCRT:utility.obj
 0002:000021f4       $unwind$__scrt_uninitialize_crt 00000001800061f4     MSVCRT:utility.obj
 0002:000021f4       $unwind$_onexit            00000001800061f4     MSVCRT:utility.obj
 0002:000021fc       $unwind$nsk_lverify        00000001800061fc     libbytecodes001.obj
 0002:0000220c       $unwind$nsk_vprintf        000000018000620c     libbytecodes001.obj
 0002:0000221c       $unwind$nsk_printf         000000018000621c     libbytecodes001.obj
 0002:00002224       $unwind$?nsk_jni_lverify@@YAHHPEAUJNIEnv_@@HQEBDH1ZZ 0000000180006224     libbytecodes001.obj
 0002:00002238       $unwind$?nsk_jni_check_exception@@YAHPEAUJNIEnv_@@QEBDH@Z 0000000180006238     libbytecodes001.obj
 0002:00002254       $unwind$Java_nsk_jvmti_unit_FollowReferences_FollowRefObjects_resetTags 0000000180006254     libbytecodes001.obj
 0002:00002254       $unwind$addRefToVerify     0000000180006254     libbytecodes001.obj
 0002:00002254       $unwind$nsk_jvmti_resetAgentData 0000000180006254     libbytecodes001.obj
 0002:00002254       $unwind$__scrt_initialize_default_local_stdio_options 0000000180006254     MSVCRT:default_local_stdio_options.obj
 0002:00002254       $unwind$?dllmain_crt_dispatch@@YAHQEAUHINSTANCE__@@KQEAX@Z 0000000180006254     MSVCRT:dll_dllmain.obj
 0002:00002254       $unwind$DllMain            0000000180006254     MSVCRT:dll_dllmain_stub.obj
 0002:00002254       $unwind$__GSHandlerCheck   0000000180006254     MSVCRT:gshandler.obj
 0002:00002254       $unwind$?__scrt_uninitialize_thread_safe_statics@@YAXXZ 0000000180006254     MSVCRT:thread_safe_statics.obj
 0002:00002254       $unwind$__scrt_acquire_startup_lock 0000000180006254     MSVCRT:utility.obj
 0002:00002254       $unwind$__scrt_dllmain_after_initialize_c 0000000180006254     MSVCRT:utility.obj
 0002:00002254       $unwind$__scrt_dllmain_before_initialize_c 0000000180006254     MSVCRT:utility.obj
 0002:00002254       $unwind$__scrt_dllmain_crt_thread_attach 0000000180006254     MSVCRT:utility.obj
 0002:00002254       $unwind$__scrt_dllmain_crt_thread_detach 0000000180006254     MSVCRT:utility.obj
 0002:00002254       $unwind$__scrt_dllmain_uninitialize_c 0000000180006254     MSVCRT:utility.obj
 0002:00002254       $unwind$__scrt_dllmain_uninitialize_critical 0000000180006254     MSVCRT:utility.obj
 0002:00002254       $unwind$atexit             0000000180006254     MSVCRT:utility.obj
 0002:0000225c       $unwind$nsk_jvmti_lverify  000000018000625c     libbytecodes001.obj
 0002:00002270       $unwind$exitOnError        0000000180006270     libbytecodes001.obj
 0002:00002280       $unwind$Java_nsk_share_jvmti_ArgumentHandler_getAgentOptionsString 0000000180006280     libbytecodes001.obj
 0002:00002294       $unwind$Java_nsk_jvmti_unit_FollowReferences_FollowRefObjects_getTag 0000000180006294     libbytecodes001.obj
 0002:00002294       $unwind$Java_nsk_share_jvmti_DebugeeClass_checkStatus 0000000180006294     libbytecodes001.obj
 0002:00002294       $unwind$agentThreadWrapper 0000000180006294     libbytecodes001.obj
 0002:000022a4       $unwind$startAgentThreadWrapper 00000001800062a4     libbytecodes001.obj
 0002:000022c0       $unwind$syncDebuggeeStatus 00000001800062c0     libbytecodes001.obj
 0002:000022c0       $unwind$__scrt_dllmain_exception_filter 00000001800062c0     MSVCRT:utility.obj
 0002:000022d4       $unwind$Java_nsk_share_jvmti_DebugeeClass_resetAgentData 00000001800062d4     libbytecodes001.obj
 0002:000022dc       $unwind$MA_checkStatus     00000001800062dc     libbytecodes001.obj
 0002:000022f0       $unwind$Java_nsk_jvmti_unit_FollowReferences_FollowRefObjects_setTag 00000001800062f0     libbytecodes001.obj
 0002:00002308       $unwind$Java_nsk_jvmti_unit_FollowReferences_FollowRefObjects_addRefToVerify 0000000180006308     libbytecodes001.obj
 0002:00002324       $unwind$checkMeth          0000000180006324     libbytecodes001.obj
 0002:00002338       $unwind$capture_previous_context 0000000180006338     MSVCRT:gs_report.obj
 0002:00002344       $unwind$__GSHandlerCheckCommon 0000000180006344     MSVCRT:gshandler.obj
 0002:00002350       $xdatasym                  0000000180006350     MSVCRT:amdsecgs.obj
 0002:00002354       $unwind$?dllmain_crt_process_attach@@YAHQEAUHINSTANCE__@@QEAX@Z 0000000180006354     MSVCRT:dll_dllmain.obj
 0002:00002390       $unwind$?fin$0@?0??dllmain_crt_process_attach@@YAHQEAUHINSTANCE__@@QEAX@Z@4HA 0000000180006390     MSVCRT:dll_dllmain.obj
 0002:00002390       $unwind$?fin$0@?0??dllmain_crt_process_detach@@YAH_N@Z@4HA 0000000180006390     MSVCRT:dll_dllmain.obj
 0002:00002390       $unwind$?fin$1@?0??dllmain_crt_process_detach@@YAH_N@Z@4HA 0000000180006390     MSVCRT:dll_dllmain.obj
 0002:00002398       $unwind$?dllmain_crt_process_detach@@YAH_N@Z 0000000180006398     MSVCRT:dll_dllmain.obj
 0002:000023ec       $unwind$?dllmain_dispatch@@YAHQEAUHINSTANCE__@@KQEAX@Z 00000001800063ec     MSVCRT:dll_dllmain.obj
 0002:00002414       $unwind$?filt$0@?0??dllmain_dispatch@@YAHQEAUHINSTANCE__@@KQEAX@Z@4HA 0000000180006414     MSVCRT:dll_dllmain.obj
 0002:0000241c       $unwind$_DllMainCRTStartup 000000018000641c     MSVCRT:dll_dllmain.obj
 0002:0000242c       $unwind$__scrt_is_nonwritable_in_current_image 000000018000642c     MSVCRT:utility.obj
 0002:0000244c       $unwind$__scrt_is_nonwritable_in_current_image$filt$0 000000018000644c     MSVCRT:utility.obj
 0002:00002454       $unwind$__scrt_fastfail    0000000180006454     MSVCRT:utility_desktop.obj
 0002:00002464       $unwind$__security_init_cookie 0000000180006464     MSVCRT:gs_support.obj
 0002:00002470       $unwind$__isa_available_init 0000000180006470     MSVCRT:cpu_disp.obj
 0002:00002480       $xdatasym                  0000000180006480     MSVCRT:guard_dispatch.obj
 0002:00002488       $xdatasym                  0000000180006488     MSVCRT:guard_xfg_dispatch.obj
 0002:00002490       .edata                     0000000180006490     bytecodes001.exp
 0002:000024b8       rgpv                       00000001800064b8     bytecodes001.exp
 0002:000024f4       rgszName                   00000001800064f4     bytecodes001.exp
 0002:00002530       rgwOrd                     0000000180006530     bytecodes001.exp
 0002:0000254e       szName                     000000018000654e     bytecodes001.exp
 0002:0000255f       $N00001                    000000018000655f     bytecodes001.exp
 0002:0000256e       $N00002                    000000018000656e     bytecodes001.exp
 0002:0000257b       $N00003                    000000018000657b     bytecodes001.exp
 0002:000025aa       $N00004                    00000001800065aa     bytecodes001.exp
 0002:000025ef       $N00005                    00000001800065ef     bytecodes001.exp
 0002:0000262c       $N00006                    000000018000662c     bytecodes001.exp
 0002:00002674       $N00007                    0000000180006674     bytecodes001.exp
 0002:000026b4       $N00008                    00000001800066b4     bytecodes001.exp
 0002:000026f1       $N00009                    00000001800066f1     bytecodes001.exp
 0002:0000272c       $N00010                    000000018000672c     bytecodes001.exp
 0002:0000275a       $N00011                    000000018000675a     bytecodes001.exp
 0002:0000278b       $N00012                    000000018000678b     bytecodes001.exp
 0002:000027ba       $N00013                    00000001800067ba     bytecodes001.exp
 0002:000027e9       $N00014                    00000001800067e9     bytecodes001.exp
 0002:0000281e       $N00015                    000000018000681e     bytecodes001.exp
 0002:00002c2a       .idata$6                   0000000180006c2a     kernel32:KERNEL32.dll
 0002:00002c8e       .idata$6                   0000000180006c8e     vcruntime:VCRUNTIME140.dll
 0002:00002dfa       .idata$6                   0000000180006dfa     ucrt:api-ms-win-crt-runtime-l1-1-0.dll
 0002:00002e1c       .idata$6                   0000000180006e1c     ucrt:api-ms-win-crt-stdio-l1-1-0.dll
 0002:00002e3c       .idata$6                   0000000180006e3c     ucrt:api-ms-win-crt-string-l1-1-0.dll
 0003:00000000       m0                         0000000180007000     libbytecodes001.obj
 0003:00000005       m1                         0000000180007005     libbytecodes001.obj
 0003:00000008       m2                         0000000180007008     libbytecodes001.obj
 0003:00000010       ?codeAttributeName@@3PEBDEB 0000000180007010     libbytecodes001.obj
 0003:00000018       ?lineNumberAttributeName@@3PEBDEB 0000000180007018     libbytecodes001.obj
 0003:00000020       ?localVarAttributeName@@3PEBDEB 0000000180007020     libbytecodes001.obj
 0003:00000028       ?localVarTypeAttributeName@@3PEBDEB 0000000180007028     libbytecodes001.obj
 0003:00000030       ?stackMapAttributeName@@3PEBDEB 0000000180007030     libbytecodes001.obj
 0003:00000038       ?callBytes@@3PAEA          0000000180007038     libbytecodes001.obj
 0003:0000003c       ?allocBytes@@3PAEA         000000018000703c     libbytecodes001.obj
 0003:00000040       meth_tab                   0000000180007040     libbytecodes001.obj
 0003:0001ab44       redefineAttempted          0000000180021b44     libbytecodes001.obj
 0003:0001ab48       nsk_context                0000000180021b48     libbytecodes001.obj
 0003:0001ab54       redefineSucceed            0000000180021b54     libbytecodes001.obj
 0003:0001ab58       agentFailed                0000000180021b58     libbytecodes001.obj
 0003:0001ab5c       currentAgentStatus         0000000180021b5c     libbytecodes001.obj
 0003:0001ab60       context                    0000000180021b60     libbytecodes001.obj
 0003:0001ac18       agentThread                0000000180021c18     libbytecodes001.obj
 0003:0001ac20       agentThreadProc            0000000180021c20     libbytecodes001.obj
 0003:0001ac28       agentThreadArg             0000000180021c28     libbytecodes001.obj
 0003:0001ac30       agent_data                 0000000180021c30     libbytecodes001.obj
 0003:0001ac40       jvmti_env                  0000000180021c40     libbytecodes001.obj
 0003:0001ac48       jvm                        0000000180021c48     libbytecodes001.obj
 0003:0001ac50       jni_env                    0000000180021c50     libbytecodes001.obj
 0003:0001ac58       checkStatus_func           0000000180021c58     libbytecodes001.obj
 0003:0001ac60       ?codeAttributeIndex@@3GA   0000000180021c60     libbytecodes001.obj
 0003:0001ac62       printdump                  0000000180021c62     libbytecodes001.obj
 0003:0001ac64       ?lineNumberAttributeIndex@@3GA 0000000180021c64     libbytecodes001.obj
 0003:0001ac68       ?localVarAttributeIndex@@3GA 0000000180021c68     libbytecodes001.obj
 0003:0001ac6c       ?localVarTypeAttributeIndex@@3GA 0000000180021c6c     libbytecodes001.obj
 0003:0001ac70       ?stackMapAttributeIndex@@3GA 0000000180021c70     libbytecodes001.obj
 0003:0001ac74       ?stackFrameOffset@@3GA     0000000180021c74     libbytecodes001.obj
 0003:0001ac78       ?mode@@3HA                 0000000180021c78     libbytecodes001.obj
 0003:0001ac7c       ?constantPoolSize@@3GA     0000000180021c7c     libbytecodes001.obj
 0003:0001ac80       ?orig@@3PEBEEB             0000000180021c80     libbytecodes001.obj
 0003:0001ac88       ?gen@@3PEAEEA              0000000180021c88     libbytecodes001.obj
 0003:0001ac90       ?inputPos@@3PEAEEA         0000000180021c90     libbytecodes001.obj
 0003:0001ac98       ?endPos@@3PEBEEB           0000000180021c98     libbytecodes001.obj
 0003:0001aca0       ?genPos@@3PEAEEA           0000000180021ca0     libbytecodes001.obj
 0003:0001aca8       ?markPos@@3PEAEEA          0000000180021ca8     libbytecodes001.obj
 0003:0001acb0       ?constantPool@@3PEAPEADEA  0000000180021cb0     libbytecodes001.obj
 0003:0001acb8       ?constantPoolCount@@3GA    0000000180021cb8     libbytecodes001.obj
 0003:0001acbc       ?zeroBytes@@3PAEA          0000000180021cbc     libbytecodes001.obj
 0003:0001acc0       ?codeLength@@3IA           0000000180021cc0     libbytecodes001.obj
 0003:0001acc4       result                     0000000180021cc4     libbytecodes001.obj
 0003:0001acc8       ?map@@3PEAIEA              0000000180021cc8     libbytecodes001.obj
 0003:0001acd0       ?widening@@3PEACEA         0000000180021cd0     libbytecodes001.obj
 0003:0001acd8       jvmti                      0000000180021cd8     libbytecodes001.obj
 0003:0001ace0       caps                       0000000180021ce0     libbytecodes001.obj
 0003:0001ad00       GS_ExceptionRecord         0000000180021d00     MSVCRT:gs_report.obj
 0003:0001ada0       GS_ContextRecord           0000000180021da0     MSVCRT:gs_report.obj
 0003:0001b270       ?g_tss_cv@@3U_RTL_CONDITION_VARIABLE@@A 0000000180022270     MSVCRT:thread_safe_statics.obj
 0003:0001b278       ?g_tss_event@@3PEAXEA      0000000180022278     MSVCRT:thread_safe_statics.obj
 0003:0001b280       ?g_tss_mutex@@3U_RTL_CRITICAL_SECTION@@A 0000000180022280     MSVCRT:thread_safe_statics.obj
 0003:0001b2a8       ?g_sleep_condition_variable_cs@@3P6AHPEAU_RTL_CONDITION_VARIABLE@@PEAU_RTL_CRITICAL_SECTION@@K@ZEA 00000001800222a8     MSVCRT:thread_safe_statics.obj
 0003:0001b2b0       ?g_wake_all_condition_variable@@3P6AXPEAU_RTL_CONDITION_VARIABLE@@@ZEA 00000001800222b0     MSVCRT:thread_safe_statics.obj
 0003:0001b2bc       ?__proc_attached@@3HA      00000001800222bc     MSVCRT:dll_dllmain.obj
 0003:0001b2d0       ?is_initialized_as_dll@@3_NA 00000001800222d0     MSVCRT:utility.obj
 0003:0001b2d1       ?module_local_atexit_table_initialized@@3_NA 00000001800222d1     MSVCRT:utility.obj
 0003:0001b2d8       ?module_local_atexit_table@@3U_onexit_table_t@@A 00000001800222d8     MSVCRT:utility.obj
 0003:0001b2f0       ?module_local_at_quick_exit_table@@3U_onexit_table_t@@A 00000001800222f0     MSVCRT:utility.obj
